:020000000F28C7
:10000800FE00030EF1000408F2000A08F300831250
:100018007F08F4006B2A1028F801D1018301D9293F
:1000280083122908AF002A08B0002B08B10003107A
:10003800300D310DB2003208B300B308031D2B2870
:100048000030A9000030AA000030AB0008002C08DE
:10005800AF002D08B0002E08B1000310300D310D8F
:10006800B2003208B800B808031D41280030A900C2
:100078000030AA000030AB00080038087B3EAF0013
:100088002F08B3072908AF002A08B0002B08B100D1
:1000980010300310B10CB00CAF0CFF3E031D4D28FF
:1000A8002F08B2003208B8002C08AF002D08B000A5
:1000B8002E08B10010300310B10CB00CAF0CFF3E8D
:1000C800031D5F282F08B2003208B8068030AF0041
:1000D8002F08B805AA17AD17FF30AC05FF30AD05DE
:1000E8000030AE050030B4000030B5000030B60076
:1000F8000730AF002F08B700291C90282C08B40738
:100108002D08031103182D0A031DB5072E08031126
:1001180003182E0A031DB60701300310AB0CAA0CF6
:10012800A90CFF3E031D912801300310AC0DAD0D45
:10013800AE0DFF3E031D99280130B702031D80282C
:100148000930AF002F08B700291CB8282C08B407BD
:100158002D08031103182D0A031DB5072E080311D6
:1001680003182E0A031DB60701300310AB0CAA0CA6
:10017800A90CFF3E031DB92801300310B60CB50CBD
:10018800B40CFF3E031DC1280130B702031DA82887
:100198003408A0003508A1003608A2003308AF00D3
:1001A8002F08A3003808B0003008A400702183127B
:1001B8002008A9002108AA002208AB000800831221
:1001C8003908BD003A08BE003B08BF0003103E0DC9
:1001D8003F0DC0004008C600C608031DFC280030BB
:1001E800BC000030BB000030BA000030B900080085
:1001F8003908BD003A08BE003B08BF00173003109D
:10020800BF0CBE0CBD0CFF3E031D03293D08C000FA
:100218004008C100BA17FF30B905FF30BA050030F1
:10022800BB053908C2003A08C3003B08C400C50131
:100238008E30C602C61F3E294608803A8F3E0318F4
:100248002E290030BC000030BB000030BA0000305E
:10025800B900080001300310C50CC40CC30CC20C53
:10026800FF3E031D2F290130BD003D08C6070319B5
:1002780059292E2918304602031C56290030BC0083
:100288000030BB000030BA000030B900080001306F
:10029800BD000310C20DC30DC40DC50DBD0B4D2906
:1002A8000130C602C608031D4B29410803196729F6
:1002B800C209C309C409C509C20A0319C30A031933
:1002C800C40A0319C50A4508BC004408BB00430812
:1002D800BA004208B90008008312230803197929D3
:1002E800220821042004031D8C290030A0000030BE
:1002F800A1000030A20008000130F5007508A3072E
:1003080001300310A20CA10CA00CFF3E031D85298F
:10031800FE3022050319A72980290130F500750848
:10032800A3070130A007003003180130A1070030EF
:1003380003180130A20701300310A20CA10CA00C75
:10034800FF3E031DA029FF3022050319B629912974
:100358000130A30201300310A00DA10DA20DFF3E34
:10036800031DAF29A11FAC292318C029FF30A00500
:100378007F30A105FF30A2050310A30C2308F50068
:10038800F601F70110300310F50DF60DF70DFF3EDD
:10039800031DC7297508A0047608A1047708A204DC
:1003A800240803190800A21708008312CF01D001FE
:1003B800CE01CB01CC01CD01CD0A8A228312851949
:1003C800EB2985148516CD01CF01D001CE01CD08CA
:1003D800031D2F2A5108013A031DFB29D1010130C1
:1003E800CF070318D00A0030D00704308506023042
:1003F8005002583003194F02031C0B2ACE08031D64
:100408000B2ACF01D001CE01CE0A8510851200300B
:100418005002053003194F02031CE2294E08013A25
:10042800031DE229322283124808CC01CC07470871
:10043800CB01CB070C304C02E53003194B02031CEF
:10044800292ACD01CD0A05152B2A85148516CF0139
:10045800D001CE01E22905158510E2298312C901D0
:10046800CA019F149F18362A1E08CA01CA07831694
:100478001E088312C901C9074A08A601A607490828
:10048800A501A507A42283122508AC002608AD0003
:100498002708AE004230A9009C30AA004030AB00CB
:1004A800142083122908B9002A08BA002B08BB00B7
:1004B800E32083123A08CA01CA073908C901C907E3
:1004C8004A08C801C8074908C701C70708008B1AA6
:1004D8000B1D7F2A643078020318772A0130F00058
:1004E8007008F8077C2AF8010130F0007008D10084
:1004F800B23081000B117408FF0073088A0072087B
:100508008400710E8300FE0E7E0E09008B0171308F
:1005180083168F00813083129F00073099000730BF
:1005280083168100B230831281000930831685005A
:1005380071309F00043083128500E0308B00080082
:1005480083122508A0002608A100A2018E30A80069
:100558002808A300A401702183122008A5002108FF
:08056800A6002208A70008000C
:02400E00C4F3F9
:00000001FF
